:10000000830100308A000428203084002A30182020
:1000100083010730BC00EF30BB002A3084003B3046
:100020001C2083010A128A11662F04068001840AAB
:100030000406031D15280034F0000A128A112C2032
:100040000A128A118000840A040870060319003419
:100050001D2883120313BB00BC1B37283C1B3F2801
:100060003C088A003B08BB0A0319BC0A82008313C0
:0E0070003C1883173B08BB0A840000080800F8
:100E98008301A500A301A4015E2F25082307840070
:100EA800831300080A128A11B9270A128A11A30AA1
:100EB8000319A40A2508230784008313800803194B
:100EC8000800512F0A128A119E270C300A128A1123
:100ED800D42701300A128A11D4270A128A112A301B
:100EE8004C278815762F8301A101A201812F0000CC
:100EF80000000000A10A0319A20A29082206031DFE
:100F0800872F28082106031908007B2F8301A700D3
:100F1800922FF230A8000130A9007727831203131B
:100F2800A70B8D2F080083010815000000000000A2
:100F380008110800830188018316880183120810AC
:100F480088106E308A273030880097270A308A2721
:100F58003030880097270A308A2730308800972752
:100F68000A308A2720308800972F8301A600023094
:100F78008A272608F039A00008080F3920048800BD
:100F880088100814972726080F39A000A00EF03003
:100F9800A00508080F392004880088100814972F26
:100FA8008301A50002308A272508F039A000080827
:100FB8000F392004880088100810972725080F3952
:100FC800A000A00EF030A00508080F392004880002
:100FD80088100810972F20347734773477342E34DC
:100FE8006F346C3469346D34653478342E3463343A
:080FF8006F346D342034003425
:02400E00323F3F
:00000001FF
